:020000002E2FA1
:08000800FF00030E8312031335
:10001000CC000A0ECD00040ECE008A110A12562F13
:10002000EE08031D14280800F9300000000000004D
:10003000000000000000FF3E031D15280000000026
:1000400000000000000000000000EE0B1428080073
:10005000F208031D2C28080004300000FF3E031D99
:100060002D2800000000F20B2C2808008312031337
:10007000D108D208D10A0319D20A0130D300D40121
:100080005108123A7A3003195206031D5428D1013F
:10009000D201C408C508C608C708C40A0319C50A9E
:1000A0000319C60A0319C70A5F1A0800D301D4014D
:1000B00083168C1008004030831203131F05FE00C6
:1000C0008316A801FE08031D281483125F128316ED
:1000D00028080319080083125F160800F501F601CD
:1000E000F801F901F701771A08000310F80DF90D6E
:1000F00083120313EF0DF00DF50DF60D7208760265
:10010000031D842871087502031C8D287108F502EF
:100110007208031CF603F6027814F70A7328ED013F
:100120006C086D020318080064000130EE00102016
:10013000ED0A9028FF3083120313EB008316051697
:10014000103083120505EB006B08EC0008008312E9
:1001500003130610861006118611061286126F0E02
:100160000F39F1000F30F10571180614F1188614DB
:1001700071190615F1198615F008031D06160A30C7
:10018000F200282086160A30F200282086120F304E
:100190006F05F1000A30F2002820061086100611C3
:1001A00086110612861271180614F1188614711938
:1001B0000615F1198615F008031D06160A30F2001F
:1001C000282086160A30F200282086120A30F20013
:1001D00028200800FD0183160313A001A101A2013C
:1001E000A301FD1A0800711C132983126D088316E0
:1001F000A00783126E08031C00296E0F0029022934
:100200008316A10783126F08031C09296F0F0929A0
:100210000B298316A2077008031C1129700F1129DE
:1002200013298316A3070310F40CF30CF20CF10C42
:1002300003108312ED0DEE0DEF0DF00DFD0AF12808
:1002400083160313A001A101A201A301A401A5012A
:10025000A601A701FD01FD1A08000310A40DA50DBC
:10026000A60DA70DF50DF60DF70DF80DA00DA10DBE
:10027000A20DA30D7C082302031D48297B0822023E
:10028000031D48297A082102031D48297908200204
:10029000031C59297908A0027A08031C7A0FA102CD
:1002A0007B08031C7B0FA2027C08031C7C0FA302AB
:1002B0002414FD0A2B297F308316031306058600BC
:1002C0007F30831206058600BF3083160605860040
:1002D000BF3083120605860008009A20EA01EC0868
:1002E000031D6A14DF106A08031DDF14DF1C0800F9
:1002F000FF30EE001020F530EE0010200130E0005D
:10030000D101D201C401C501C601C7015F110800B6
:10031000EB1F97292D30EF001030F000A7206A085E
:10032000003CEF00EB090318EB0A6F08EA006A08CB
:10033000EC006B08ED0027306B02031DA129103083
:100340006A02031CD129EB1BD129F3016C08EF00D1
:100350006D08F000ED1FB229EF09F009EF0A03194B
:10036000F00AF30A1030F1002730F2006E2078080E
:1003700083120313EE00731CBF29EE09EE0A6E0808
:10038000303EEF001030F000A7206E08003C03184C
:10039000D1291030EC022730031C2830ED02EE0387
:1003A000C52903306B02031DD729E8306A02031CFC
:1003B000092AEB1B092AF4016C08EF006D08F00014
:1003C000ED1FE829EF09F009EF0A0319F00AF40A12
:1003D000E830F1000330F2006E207808F300741C5E
:1003E000F329F309F30A730883120313EE006E086E
:1003F000303EEF001030F000A7206E08003C0318DC
:10040000092AE830EC020330031C0430ED02EE034D
:10041000FD296B08803AEF0080306F02031D122A1D
:1004200064306A02031C402AF4016C08EF006D0876
:10043000F000ED1F212AEF09F009EF0A0319F00A75
:10044000F40A6430F100F2016E207808F300741CA5
:100450002B2AF309F30A730883120313EE006E08C4
:10046000303EEF001030F000A7206E08003C03186B
:10047000402A6430EC02ED08031CED03EE03352A3C
:100480006B08803AEF0080306F02031D492A0A3062
:100490006A02031C772AF4016C08EF006D08F00073
:1004A000ED1F582AEF09F009EF0A0319F00AF40AC0
:1004B0000A30F100F2016E207808F300741C622A01
:1004C000F309F30A730883120313EE006E08303E3B
:1004D000EF001030F000A7206E08003C0318772AC8
:1004E0000A30EC02ED08031CED03EE036C2A6C08E5
:1004F000303EEF001030F000A7200800EB08031D8D
:10050000842A8030EB00862AC030EB006A086B0733
:10051000EF00F001A7200230EC008F2008006A08ED
:10052000EF001030F000A720080083160313061018
:100530008312061083168610831286108316061106
:1005400083120611831686118312861183160612F2
:100550008312061283168612831286120C30EC0068
:100560008F203330EF00F001A7200230EC008F2005
:100570003330EF00F001A7200230EC008F20323042
:10058000EF00F001A7200230EC008F202C30EF00AC
:10059000F001A7200230EC008F200630EF00F001C0
:1005A000A7200230EC008F200C30EF00F001A720D4
:1005B0000230EC008F200130EF00F001A720023064
:1005C000EC008F200230EF00F001A7200230EC0099
:1005D0008F2008000730831203139F00C03083165A
:1005E00081009522B801B901BA01BB01C001C10166
:1005F000C201C301D101D201C401C501C601C701B5
:10060000073083168500063083129F00EF30831673
:100610009F008B1783120C1383160C170B178B1765
:100620006D216003031D5F2B0B1712109210121522
:1006300007301205EA0020306A0492000F3083165A
:1006400092008B178C1483125F19432B4030831652
:1006500006048600403083120605EA00EB014030B4
:100660006A020319EB0A5F106B08031D5F147F30E9
:100670008316060586007F3083120605EA00803067
:100680006A0486005F2B8030831606048600803063
:1006900083120605EA00EB0180306A020319EB0AB7
:1006A0005F106B08031D5F14BF30831606058600BC
:1006B000BF3083120605EA0040306A0486005F1AE4
:1006C000ED2DEC015F19652BEC0AEA012330510294
:1006D000520803186D2B0319EA0A6A08EC05EB01AE
:1006E000EB0AC408031D6B10C508031D6B10C60878
:1006F000031D6B10C708031D6B106B086C050319F5
:100700008B2B5F150130E000DE00D101D201C40166
:10071000C501C601C7015F1D7A2C5E03031D9B2B1B
:100720005B21FF30EE001020F530EE001020DE01DE
:100730005F155F16ED2D5B21FF30EE001020F530C8
:10074000EE001020403083160604860040308312ED
:100750000605ED00EE0140306D020319EE0A5F1050
:100760006E08031D5F14E0014408ED004508EE002B
:100770004608EF004708F0001230F1007A30F2002E
:10078000F301F401EA20831620088312C4008316C3
:1007900021088312C500831622088312C60083161F
:1007A00023088312C7005108ED005208EE00EF0144
:1007B000F00144086D07BC004508BD006E08031831
:1007C0006E0FBD074608BE006F0803186F0FBE0707
:1007D0004708BF0070080318700FBF073C08ED0002
:1007E0003D08EE003E08EF003F08F000E430F10065
:1007F0002530F200F301F401EA2083162008F50009
:100800002108F6002208F7002308F8001230F9004A
:100810007A30FA00FB01FC01202124088312C80071
:10082000831625088312C900831626088312CA007E
:10083000831627088312CB000130C8020030FD0068
:10084000031C7D0FC9020030FD00031C7D0FCA028E
:100850000030FD00031C7D0FCB024808F50049085D
:10086000F6004A08F7004B08F8006430F900FA0176
:10087000FB01FC01202124088312B80083162508FF
:100880008312B900831626088312BA00831627083C
:100890008312BB003808ED003908EE003A08EF007B
:1008A0003B08F0006430F100F201F301F401EA20AA
:1008B00083162008F5002108F6002208F700230817
:1008C000F800750883124802C0004908C1004A08B0
:1008D000C2004B08C3007608031C760FC1027708DC
:1008E000031C770FC2027808031C780FC302013083
:1008F000E100ED2D5B21FF30EE001020F530EE0021
:10090000102080308316060486008030831206058E
:10091000ED00EE0180306D020319EE0A5F106E08E3
:10092000031D5F14E0014408ED004508EE00460891
:10093000EF004708F0001230F1007A30F200F301C6
:10094000F401EA2083162008F5002108F6002208A9
:10095000F7002308F80083125108BC005208BD00BC
:10096000BE01BF017508BC0776080318760FBD07E6
:1009700077080318770FBE0778080318780FBF07AA
:100980003F08003C031DCE2C3E08003C031DCE2C2E
:100990003D087D3C031DCE2C3C08003C03186A2D0D
:1009A0003C08F5003D08F6003E08F7003F08F80057
:1009B0000A30F900FA01FB01FC012021240883120E
:1009C000B400831625088312B50083162608831207
:1009D000B600831627088312B7003408ED003508E7
:1009E000EE003608EF003708F000CA30F10003309F
:1009F000F200F301F401EA2083162008F500210833
:100A0000F6002208F7002308F8003530F9000C3012
:100A1000FA00FB01FC01202124088312C800831680
:100A200025088312C900831626088312CA0083167C
:100A300027088312CB004808F5004908F6004A0849
:100A4000F7004B08F800E830F9000330FA00FB012A
:100A5000FC01202124088312B80083162508831284
:100A6000B900831626088312BA008316270883125A
:100A7000BB003808ED003908EE003A08EF003B08EB
:100A8000F000E830F1000330F200F301F401EA2055
:100A900083162008F5002108F6002208F700230835
:100AA000F800750883124802C0004908C1004A08CE
:100AB000C2004B08C3007608031C760FC1027708FA
:100AC000031C770FC2027808031C780FC302DF15DE
:100AD000E101ED2D3C08B4003D08B5003E08B6002C
:100AE0003F08B7003408ED003508EE003608EF0087
:100AF0003708F000E430F1002530F200F301F40192
:100B0000EA2083162008F5002108F6002208F700E5
:100B10002308F8003530F9000C30FA00FB01FC0125
:100B2000202124088312C800831625088312C900D7
:100B3000831626088312CA00831627088312CB0067
:100B40004808F5004908F6004A08F7004B08F80085
:100B50006430F900FA01FB01FC0120212408831212
:100B6000B800831625088312B9008316260883125D
:100B7000BA00831627088312BB003808ED00390835
:100B8000EE003A08EF003B08F0006430F100F2019B
:100B9000F301F401EA2083162008F5002108F6008D
:100BA0002208F7002308F800750883124802C000E5
:100BB0004908C1004A08C2004B08C3007608031C5C
:100BC000760FC1027708031C770FC2027808031C56
:100BD000780FC302DF110130E1006430EE00102015
:100BE0000130EA00EB017E224330EA008F22203000
:100BF000EA008F223D30EA008F222030EA008F2267
:100C00003808EA003908EB0088212E30EA008F22EC
:100C1000E30100304302031D172E00304202031D82
:100C2000172E00304102031D172E0A304002031C0C
:100C3000E30AE20161030319E20A6208630503198A
:100C4000242E3030EA008F22E60100304302031DDB
:100C5000332E00304202031D332E00304102031DAB
:100C6000332E64304002031CE60AE40100304302E4
:100C7000031D442E00304202031D442E0030410269
:100C8000031D442E0A304002031CE40A6408E605F2
:100C9000E501E50AE108031D65106508660503190D
:100CA000572E3030EA008F223030EA008F22E901DF
:100CB00000304302031D662E00304202031D662EE3
:100CC00000304102031D662E64304002031CE90A15
:100CD000E7014308003C031D772E4208003C031D3A
:100CE000772E4108003C031D772E40080A3C031C68
:100CF000E70A6708E905E801E80AE108031D68104A
:100D0000680869050319872E3030EA008F224008F1
:100D1000EA004108EB0088215F1DA12E2030EA0087
:100D20008F226E30EA008F224630EA008F22203078
:100D3000EA008F222030EA008F222030EA008F2242
:100D4000C82EDF1DB62E2030EA008F226D30EA005B
:100D50008F224630EA008F222030EA008F22203096
:100D6000EA008F222030EA008F22C82E2030EA00CD
:100D70008F227530EA008F224630EA008F22203021
:100D8000EA008F222030EA008F222030EA008F22F2
:100D90000130EA00EB007E220130530603195408AB
:100DA000031DFD2E2030EA008F222030EA008F2222
:100DB0002030EA008F222030EA008F222030EA0023
:100DC0008F225430EA008F224530EA008F225330C0
:100DD000EA008F225430EA008F222030EA008F226E
:100DE0002030EA008F222030EA008F222030EA00F3
:100DF0008F222030EA008F22102B2030EA008F2231
:100E00002030EA008F222030EA008F222030EA00D2
:100E10008F222030EA008F222030EA008F222030FB
:100E2000EA008F222030EA008F222030EA008F2251
:100E30002030EA008F222030EA008F222030EA00A2
:100E40008F222030EA008F222030EA008F222030CB
:100E5000EA008F222030EA008F22102BD530831237
:100E60000313A000C430A100BB30A200DC30A300FB
:100E7000A401A501A601A701A801A901AA01AB012E
:100E8000AC01AD01AE01AF01D801D901CF01D00154
:100E9000DA01DB01DC01DD01B001B101B201B30116
:100EA000D601D701D5018A110A12EA2A8312031347
:100EB0000C1F5D2F5B2083120C138C1C652F831677
:100EC0008C1C652F362083128C1083124E0E8400EA
:0E0ED0004D0E8A004C0E8300FF0E7F0E0900AF
:02400E000A3F67
:00000001FF
